:080000007522001200F2013329
:20000B00C2A9C28CDF013230BC08758C51758A00012E201208758CF9758A00012E758CFF34
:20002B00758A40D28CD2A932E47821F6D8FD75810812280ED2AF12004B1201260133014150
:20004B00C210C212C2BC7B0275260012007FF52704F9782B12007FF6082526F526D9F51237
:20006B00007FB526067455120092227401120092DBD60133900000209808A3AC83BCFFF7B4
:20008B000133E599C298223099FDC299F599227B02752600782BAE27E527141200927F146F
:2000AB00DFFEE6081200927F14DFFE2526F526DEF1E5261200927F14DFFE12007FB4550167
:2000CB0022DBCE0133752B5575270112009A22752B0101D33099FDC299D299201B29201A17
:2000EB001E20191320180875CBFF75CAB8211575CBFF75CAF4211575CBFF75CAFA21157514
:20010B00CBFF75CAFD211575CBFF75870075984075890175C834D2CAD29C22852B25852CEE
:20012B0018852D1B852D23852E1A852F1985301E85311D85321CC211E52530E602D211C24D
:20014B00E6F525E518543F902D6593FDE51854C07002D2BC30E704D212C2BCE518543FB480
:20016B000E06D2BA740A2190B42104D2112190B43504D2112190B42202D211B43D02D21126
:20018B00B43E02D211FAE525540FB40003C21022B40103020DFAB40205D210021921B4031A
:2001AB0005D213020DFAB4040201DFB40503020FFCB40605D214020DFAB40705D217020D78
:2001CB00FAB40803022188B4090302301CB40A03022EC9B40B03022EFBB40C03022EF0B464
:2001EB000D030201F2013375F68775F65975BF0375880075B80075A8827EF07FFF8E8A8F72
:20020B008C7F007589017588107587017901BA0A0279057F0EDFFE123067D9F722C213BA6D
:20022B001264121C31120F047519FF751AFF121C607EFC121C761228AC1227C5122834752B
:20024B00F020121C9B7F0EDFFE431F801228447F0312223C531F7F1228447F0EDFFED294BF
:20026B00121C741227C55321F712283475F020121C9B7F0EDFFEC2947F0EDFFE1227C51272
:20028B0028341200D022D2B3D2B5D294BA0A08301D03020412D2951228AC301E30D284D25A
:2002AB00A3D283301806C284712C614930180CC284712CD284C2A3712C6149C284712CD272
:2002CB0084C2A3712CD2A3C283712C614930180451FF614930190B51FF7F6412223C7117C7
:2002EB00614951FF7F6412223C71177F6412223C712C61491227C5122834531F7F122844A9
:20030B007420121CAA1202171227E2221227E2431F801228447420121CAA1202171227DBD8
:20032B00221227C55321F7122834C2B3531F7F1228447420121CAA1202171227DB22121CDA
:20034B00A8C2941200D022C21774FF7EFF1223F17526007B021228A1122897D2B7D28612EA
:20036B002588D3920E1228347401121CAAD28012258874007E901223F112503074FF7EFF5C
:20038B001223F1122588C286C2B7122401CED2B7D286020FE4B4FF10EEB4FF0C12285230A5
:2003AB00102C1200D0020ED61200DA020ED620179674FF7EFF1223F17526007B021228A186
:2003CB0012289774FF7EFF1223F1C2B7D2801225881224012014BE1200922526F526EE126E
:2003EB0000922526F5261228523010E2E52612009212007FB45503020ED8852D1B852E1A7E
:20040B00852F19DBC901331228ACC291122897D280D29730181ED286D2B2D290D285D2D9C1
:20042B00C2DA121CA47F14C29712223CD297121CA802045AD286D2B2C290C285D2D9C2DA8C
:20044B00121CA47F14C29712223CD297121CA87E0020D90512176DDEF861491228ACC29159
:20046B00122897D280D297D286C2B2C290C285D2D9C2DA121CA47F28C29712223CD297127C
:20048B001CA8021441C291122897D297C286D2B2D290D285D2D9C2DAD280123B841200D0D8
:2004AB0012220D782B12071C121CA47F01C29712223CD297121CA87E0020D90812176D1297
:2004CB00176DDEF5C2B2D2B2122852D2DA0000C2DA08D527D01200D03010C5020ED8A28425
:2004EB0092E0A2A392E1A28392E2A2A292E3A28292E4A28192E5A2A192E6A2A092E7223079
:20050B001303020228301703020FA6C291122897C2DAD280D297D285D290C2B2C286123B50
:20052B00841204E9301406B4FF2F02053F1200922526F526122852D2DA0000C2DA3010E1BC
:20054B00301473020F22E519C4035407F5F0E51AC454F00345F0F5F0221200DA020ED63059
:20056B0013030206EC3017030206B51205CA120607120551120693D285D290C2B2C28612C5
:20058B0004E9301406B4FFD102059D1200922526F526122852D2DA0000C2DAE519541FB4EE
:2005AB00000B120693D285D290C2B2C2863010CF301403020F22E52612009212007F221208
:2005CB001C74C291C2DA1228A1122897121C9012176D12176D1228AC12176D12176DD28097
:2005EB007B14121C92D297D285D290C2B2D28612176D12176D12176D12176D22121CA41255
:20060B00176D12176D12176D12176D221205CA120607D286C2B2C290C28512176DD2D97F42
:20062B0028C29712223CD297121CA80214411205CA12060712055112176D12176D12176DFE
:20064B00D2D91200D012220D120693D285D290D2B2C28612176D782B12071CC29712176D34
:20066B00D297122852D2DA0000C2DA08D527E97E0020D90812176D12176DDEF51200D030B5
:20068B0010C3121CA8020ED812176DD285D290C2B2D28612176DE5F005F012071DD2DA0061
:2006AB0000C2DA12176D121C7422C2171205CA120607120551E5F0B4000BC290C285D28673
:2006CB00D2B20206E6120693E51930E006D2DA0000C2DAD285C290C2B2C2861204E9020F21
:2006EB00E4C2131205CA120607D285D290D2B2D28612176DD2D9E51912071DC29712176D3D
:20070B00D2977F2812223C7B28121C92121CA86149E6A2E09284A2E192A3A2E29283A2E317
:20072B0092A2A2E49282A2E59281A2E692A1A2E792A022B4FF10EEB4FF0C12285230103939
:20074B001200D0020ED61200DA020ED6D2B4D2B2D2B3D2840000C2840000D28412176D12CB
:20076B00176D12176D12176D12176D12176DC2B2C2B374FF7EFF1224F4C2B2C2B312251F50
:20078B001225082014AD1200922526F526EE1200922526F5261228523010DEE526120092D3
:2007AB0012007FB45503020ED8852D1B852E1A852F19DBC50133B4FF10EEB4FF0C12285272
:2007CB003010461200D0020ED61200DA020ED6D2B4D2B2D2B3D2840000C2840000D284125B
:2007EB00176D12176D12176D12176D12176D12176DC2B2C2B3E51BA2E6920CA2E7920D1233
:20080B00283474FF7EFF1224F4C2B2C2B312251F1225082014A01200922526F526EE1200FB
:20082B00922526F5261228523010DEE52612009212007FB45503020ED8852D1B852E1A85B8
:20084B002F19DBC50200331228A112289712176DD2A5D2A2D2A3C2B5C2B3D2A1D2A422C314
:20086B00E519241FF519E51A3400F51AE51B3400F51BE51CB5190DE51DB51A08E51EB51B10
:20088B0003D21022C3E5192401F519E51A3400F51AE51B3400F51B22E51E30E7030209FD85
:2008AB007526001208523017030209B774001209871208D730A3FD1208FA12086A3010EC7F
:2008CB00E52612009212007F12280E22C2A1D2B3E519F590C2A5D2A5C2A1D2B3E51AF590AE
:2008EB00C2A5D2A5E51BF590C2A5D2A5C2B3227F20C2A174FFF590C2A2E590D2A21200922A
:20090B002526F526DFF1D2A122E51E30E703020AD0C2101208521200D012220D7480120998
:20092B00871208D7120950741012098730A3FD12099420E00D12086A3010DB1200D012285C
:20094B000E22021CC37F20C2A1782BE6F590C2A5D2A508DFF622E51E20E703020B1D12083D
:20096B0052C2A174601209871208E374D012098730A3FDD2A11200D012280E22C2A1D2B5E5
:20098B00F590C2A5D2A5C2B522C2A1747012098774FFF590C2A200E590D2A2D2A122C3E5E5
:2009AB001A3401F51AE51B3400F51B22C217752600120852C2A1749012098700D2B3007486
:2009CB0000F590C2A500D2A500C2B30074FFF590C2A2E590D2A21200922526F526C2A2E59C
:2009EB0090D2A2120092252612009212007F12280E227526001208522017B1AC1CC21212BD
:200A0B000A8230A3FDC2A174FFF5907B027F00C2A2E590D2A21200922526F526DFF1DBED29
:200A2B001209A9D2A1DCD8E52612009212007F12280E227526001208523017030209B7AB58
:200A4B001DAC1CEC60010BC212E51E120987120A8230A3FDC2A174FFF590C2A2E590D2A2BF
:200A6B001200922526F526DCF1DBEFE52612009212007F12280E22C2A1D2B3E519F590C2F3
:200A8B00A5D2A5C2A1D2B3E51AF590C2A5D2A5E51BF590C2A5D2A5C2B322C2A174FFF59090
:200AAB007F00C2A2E590D2A21200922526F526DFF17F00C2A2E590D2A21200922526F526AF
:200ACB00DFF1D2A122C2101208527D047480120987120A821200D012220D120B0DDDF57420
:200AEB001012098730A3FD12099420E0121209A9E51C9404F51C70D21200D012280E2202AA
:200B0B001CC3C2A1782BE6F590C2A5D2A508D527F522120852C2A17460120987120A8E741E
:200B2B00D012098730A3FDD2A11200D012280E22C3E51A3401F51AE51B3400F51BE51E3428
:200B4B0000F51E227526001208523017030209B7E51D54F0C4FFE51D540FF51DEF704DAB6B
:200B6B001D0BAC1C7400120987120C1630A3FDC2A174FFF59020141FC2A2E590D2A2120053
:200B8B00922526F526DCF1AC1CDBEDE52612009212007F12280E22C2A2E590D2A2B4FF65E6
:200BAB00DCF5AC1CDBF11200D0020ED6C212AB1D0BAC1C7400120987120C1630A3FDC2A111
:200BCB0074FFF590201424C2A2E590D2A21200922526F526DCF1AC1CDBED120B3BDFCDE51D
:200BEB002612009212007F12280E22C2A2E590D2A2B4FF11DCF5AC1CDBF1120B3BDFAD12B9
:200C0B0000D0020ED61200DA020ED6C2A1D2B3E519F590C2A5D2A5C2A1D2B3E51AF590C2CA
:200C2B00A5D2A5E51BF590C2A5D2A5E51EF590C2A5D2A5C2B322C2101208527D0474801268
:200C4B000987120C161200D012220D120C7EDDF5741012098730A3FD12099420E012120B60
:200C6B003BE51C9404F51C70D21200D012280E22021CC3C2A1782BE6F590C2A5D2A508D5E9
:200C8B0027F522120852C2A17460120987120C2274D01209877F0512223C30A3FDD2A11257
:200CAB00099420E0071200D012280E221200DA12280E22C3E51A3401F51AE51B3400F51B99
:200CCB00227526001208523017030209B7E51DFBAC1CEC60010BC2127400120987120D327C
:200CEB00743012098730A3FDC2A174FFF59020141DC2A2E590D2A21200922526F526DCF103
:200D0B00DBEFE52612009212007F12280E22C2A2E590D2A2B4FF0ADCF5DBF31200D0020EB9
:200D2B00D61200DA020ED6C2A1D2B3E519F590C2A5D2A57400F590C2A5D2A5C2A1D2B3E513
:200D4B001AF590C2A5D2A5E51BF590C2A5D2A5C2B322C2A174FFF5907F00C2A2E590D2A2EA
:200D6B001200922526F526DFF17F00C2A2E590D2A21200922526F526DFF1D2A122C210126F
:200D8B0008527D107480120987120D321200D012220D120DBADDF5741012098730A3FD12A4
:200DAB00099420E0071200D012280E22021CC3C2A1782BE6F590C2A5D2A508D527F52212DB
:200DCB000852C2A17460120987120D4674D01209877F1412223C30A3FDD2A112099420E095
:200DEB00071200D012280E221200DA12280E22BA2E030208A3BA3C03020A3EBA3B03024822
:200E0B00F2BA37030232D0BA13030203B9BA14030203B9BA18030203B9121C747526007B75
:200E2B00021228A1122897BA2F03020757121C74902AEF022AA1D281020EA5752100D2A085
:200E4B00D284D2A4D2A1C2A4C284121C74D280020EA5121C31120F04020E9C301C0302056D
:200E6B006A301D0302050A121C90D290C2B3C2B5C2A5D285D2A4531F7F122844301E0F127E
:200E8B0028B31227C512283475F020121C9B020E9C121C90301303020228301703020F2754
:200EAB00121C60BA1207120EF07B3CDBFE121C512014571200922526F5261228523010DA6C
:200ECB00201454E52612009212007FC214531FFB12284412280E22852D1B852E1A852F19AD
:200EEB00DBB8020033C0E0431F801228441227C55321F7122834D0E022C0E0531F7F1228AB
:200F0B00441227C5122834D0E022B4FF0512285280AB1200DA80B41200D080AFC217752135
:200F2B0000121C601228B3902C69022AA1D2827404121CAA020FE1BA0F028003020F4D20D7
:200F4B001D2BBA24028003020F58201D20BA25028003020F63020F78BA11028003020F6EE5
:200F6B00201F0AD2837408121CAA020FE1201CF3D2857420121CAA020FE1201D1E301E08ED
:200F8B007420121CAA020F98301F02C294D2851227E2431F80122844020FE1C217C2911288
:200FAB002897C2DAD280D297C290C285C286C2B2123B84A28492E0A2A392E1A28392E2A25F
:200FCB00A292E3A28292E4A28192E5A2A192E6A2A092E7020FE4121C51F526120092E52607
:200FEB0012009212007F121CA822740080EB021441121C74902B6D022AA112109A12108E80
:20100B00D2827405121CAA02102B12109A201F0612108E0210241228B3D282740C121CAA63
:20102B00C2847F6412223CD28402144112109A201F0612108E0210461228B3D283D280D2F0
:20104B0084C2A47409121CAAC2A07F6412223CD2A0D2A402144112109A12108ED284D2833B
:20106B007409121CAA02108212109A12108ED284D2837418121CAAC2A47F6412223CD2A4D2
:20108B00021441E51F54E54402F51F122846221228A1122897121C7422C212BA17397404EF
:2010AB00122836122897201805C2A10210C13019030240D3D2A1D2B4C280D2801240C275FA
:2010CB00F040D212123FEEC2D9C280D28030B4FDD2D9C212021441BA3B0302495B1228A153
:2010EB00122897121C90BA180280030211BE301F03021138D2B7D286122588D3920E122844
:20110B003412502612504112505612502612504112506274FF7EFF1223F17D00C286C2B76A
:20112B00122401D2B7D28630E7F202144174FF7EFF1223F17526007B021228A11228971240
:20114B0028ACD2B7D286D3920E1228347401121CAAD2801225887C0074007E201223F112CA
:20116B00503074007E201223F11250307B14121C920C12258874007EA01223F112503012A4
:20118B00176D12176D74FF7EFF1223F1C286C2B7122401D2B7D286B4FF0DEEB4FF09122897
:2011AB00523010CE0214411211B780ACBC19031200DA22121C74BA122E121C31120F04E57C
:2011CB001F546544804402F51F122846D2917420121CAA7F0A12223C531F7F12284475F0F2
:2011EB0000121C9B021441BA0A02800302130D301C03020617301D03020466D2A4D290C295
:20120B00A5D2B5C2B3301F02D294121C90121CA8431F80E51F54FD122846D2857420121C07
:20122B00AA7F0EDFFE301F3B1228911228B37F96123069531FFB122844121C90431F04126C
:20124B0028447F96123069531FFB122844121C90431F04122844121CA8D29053A01FD2A40A
:20126B000214417F0A123069121CA8D290C2B3C2B5C2A5D2A4021441BA1E0280030212B25D
:20128B00D2BCD283D284D2A01228B37408121CAAC284C2A07F0112223CD2A0D28474001271
:2012AB001CAAC2BC021441BA1D0280030212DED2BC43800E1228B37404121CAAC283C28116
:2012CB007B28121C92D281D2837400121CAAC2BC021441BA100280030213B6301F12122921
:2012EB00F1122A37D2BC7F2812223CC2BC0214411229E112295AD2BC7F2812223CC2BC022F
:20130B001441D284752110122834D2A4D2A0BA1902800302133A12203A7E30121C76122A7A
:20132B007C7E30121C76122A7C121C74021388BA240280030213446166BA250280030213E1
:20134B004E6166BA0F028003021283301F0D1228B3D2807401121CAA02137F301D1612286F
:20136B00B3D2847410121CAA1229E112295A121C740213991229E112295A121C74C2A4C281
:20138B0084121C51D284D2A430E7F2021441C2A4C3920C122834121C51F5F0D3920C1228CF
:2013AB0034D2A4E5F030E7E6021441E51F54FD122846BA113F301F1A7411121CAA121C601C
:2013CB007E20121C76122A7C7ED0121C76122A7C80BCD392A17411121CAA121C607E201281
:2013EB001C76122A7C7ED0121C76122A7C121CA4D2848089121CA4301F137E30121C761225
:20140B002A7C0000122A7C121C740213887B147E20121C76122A7C0000122A7C7F0A122226
:20142B003C7EA0121C76122A7CDBE47E00121C76122A7C121CA81200D0221228A1122897CC
:20144B00D2B4D2B2D2B3D2B5D282D2840000C2840000D28412176D12176D12176D12176DCD
:20146B0012176D12176D7400F51B201F4474057E557FAA12158F74027EAA7F5512158F7467
:20148B00057E557F8012158F74057E557FAA12158F74027EAA7F5512158F74057E557F1086
:2014AB0012158F121C90121C9012250830E7F7808574557E557FAA12158F742A7EAA7F5588
:2014CB0012158F74557E557F8012158F74557E557FAA12158F742A7EAA7F5512158F745566
:2014EB007E557F1012158F121C9080BA1228A11228811228971228ACD280D2B4D2B2D2B3A3
:20150B00D2B5D2840000C2840000D284D28012176D12176D12176D12176D12176D12176D71
:20152B0012251F74607E001224F4C2B2C2B400D2B4D2B274D07E001224F4C2B2C2B400D232
:20154B00B4D2B274207E001224F4C2B2C2B400D2B4D2B274D07E001224F4C2B2C2B400D270
:20156B00B4D2B2121C90121C90121C907F32121C90D2B3D2B212250820E706DFF11200DA6E
:20158B00220214418E19F51A12251FEF7E001224F4C2B2C2B400D2B4D2B222C280C2D8C270
:2015AB00D97440121CAAC2B41216B575F0FFD21212160BE5F060211216C512176D1216B537
:2015CB00E5F0B4FF32E51BC4540FB40506E5F04401A1E074A112167012168D120092252674
:2015EB00F5261228523010F01216C5E52612009212007F12280E22E5F0440112167080D868
:20160B00E51BC4540F901616022AA216D516E416EF170117151725173C7440121CAA1200B3
:20162B00D012220D122897C280C2D8C2D9C2B4E51B540F90166993FB1216B5C21212160BEC
:20164B00782BE612167008122852DBF61216C51200D020100512220D80CD12280E220004F9
:20166B000810204080790833928100D2A112176DC2A112176DD9F0D28100D2A112176DC2B7
:20168B00A1227908D2A10000000000A281330000000000C2A10000000000D9E8C28100D2F9
:2016AB00A112176DC2A100D28122D28100D2A112176DC28112176DC2A122C28100C2A1129E
:2016CB00176DD2A112176DD28122E519C3301201D33312167075F0002274A0121670E5192A
:2016EB0012167022E51A23540E24A054FE121670E51912167022E51A23540E24A054FEF5AC
:20170B00F0121670E5191216702274A0121670E51A121670E51912167022E51B23540224E6
:20172B00A0F5F0121670E51A121670E51912167022E518035460F5F0E525548045F0C4546E
:20174B000E44A0F5F030E102D28030E202D2D830E302D2D9121670E51A121670E51912166F
:20176B00702200000000000022E52703547FF52722301F0302186F1228A1122897D2B7D2A8
:20178B0086122588D3920E12283402179B122588C2BCD212D2B7D2861200D012220D121716
:2017AB0074782B7C00D2B7D286BA1815C019C01AC01B12502612504112506ED01BD01AD095
:2017CB0019122588E6FE08E6CE1223F1BA18061250300218147401121CAABA140CC2867FDA
:2017EB000112223CD28602180FC286E5F054BFF5211228347F0112223CE5F04440F52112C7
:20180B002834D2867400121CAA0C74FF7EFF1223F1BA1814080218507D00C286C2B71224CF
:20182B0001D2B7D286021850C286C2B7122401D2B7D286F5258E1818E60886F008B5251C3E
:20184B00E5F0B51817122852D5270280030217AE20100302179B1200D0020ED812190518F7
:20186B00180217B01228A11228971228ACD2B7D286D3920E1228347401121CAAD280120077
:20188B00D012220D121774782B7C0012258874007E401223F1125030E6FE08E6CE1223F101
:2018AB0012503012176D12176D12176D12176D74007EC01223F112503012176D12176D0C91
:2018CB0074FF7EFF1223F1C286C2B7122401D2B7D286F5258E1818E60886F008B52514E5F7
:2018EB00F0B5180F122852D5279F3010911200D0020ED812190518188094BC191885252E16
:20190B0085182F752705851B2B851A2C85192D12009A02003322BA2E03020914BA3C0302E6
:20192B000AD0BA3B03024986121C7420100122C210EA9415604D14604A1460471228A1128C
:20194B0028811228971228ACBA100302198EBA1F03021979EA94216015146012BA190221A6
:20196B0079BA35022179EA9412400302198EBA0A0C301C03020639301D030204901200D0B4
:20198B0012220D902BEB022AA1D2810219D1752100D2A0D284D2A4C2A4C284D2800219D18B
:2019AB00121C31120F0421D1D290C2B3C2B5C2A5D285D2A4301F04D2B3D294531F7F1228BB
:2019CB00447B78121C92782BBA190312203A121C16BA1203120F04121C7412285208D527B6
:2019EB00ED1200D0301099020ED812176DD2B4D2B2D2B3D2B5D282D2840000C2840000D2DE
:201A0B008412176D1200D0301E03021A9B12220D782B121774C019C01AC01B7400F51B2004
:201A2B001F5174057E557FAA12158F74027EAA7F5512158F74057E557FA012158FD01BD0FC
:201A4B001AD01912251FE6FE08E608CE1224F4C2B2C2B400D2B4D2B212176D12250812175E
:201A6B006D122508122852D527AB1200D030109D020ED874557E557FAA12158F742A7EAA94
:201A8B007F5512158F74557E557FA012158F80ADC019C01A121AEED01AD01912220D782B8F
:201AAB0012177412251F74A07E001224F4C2B2C2B400D2B4D2B2E6FE08E608CE1224F4C2E4
:201ACB00B2C2B400D2B4D2B212176D12250812176D122508122852D527C91200D03010BBF1
:201AEB00020ED874057E557FAA12158F74027EAA7F5512158F74057E557F2012158F2212CB
:201B0B00176DD2B4D2B2D2B3D2B5D282D2840000C2840000D28412176DE51BA2E6920CA27C
:201B2B00E7920D1228341200D0C019C01A121AEED01AD01912220D782B12177412251F74D9
:201B4B00A07E001224F4C2B2C2B400D2B4D2B2E6FE08E608CE1224F4C2B2C2B400D2B4D22A
:201B6B00B27F6412176DDF03021CC330B5F5122852D527C81200D03010BA020ED8021CC39D
:201B8B0012176DD280D2B4D2B2D2B3D2840000C2840000D284D28012176D1200D012251FB1
:201BAB0074607E001224F4C2B2C2B400D2B4D2B274D07E001224F4C2B2C2B400D2B4D2B2CA
:201BCB0012220D782B12177412251F74407E001224F4C2B2C2B400D2B4D2B2E6FE08E608F9
:201BEB00CE1224F4C2B2C2B400D2B4D2B212176D12250812176D122508122852D527C912E1
:201C0B0000D03010BB121CA8020ED87C00121C60BA1207120EF07F28DFFE121C3D500122E1
:201C2B00902CE7022AA1D2905390E1D2A5D285C2A422121C51F5F0E6B5F002D322C322746E
:201C4B00038CF0A4FF22901C58ED022AA2226522DC23D02699901C67ED022AA2227E22FDB2
:201C6B00241026B6E6FE021C767EFF901C7DED022AA2224322BA23AE26777B017C000000C9
:201C8B00DCFCDBF8227BA07C000000DCFCDBF822E5F0021CAA742181AA740181AA74005443
:201CAB007F3011024480122AAED2A6C2A7C287D2872220BC03BC1917F52E85F02F752705D1
:201CCB00851B2B851A2C85192D12009A02003322752100D2A0D284D2A4C2A4C284D28012B1
:201CEB001C60C2BCD284D3920C122834D2A4D2A0D2801228B3D2847410121CAABA250312DD
:201D0B002A5E1200D012220D782B122A68121C60121C6F122A7C7F10DFFE121C74121C7433
:201D2B0012285208D527E33010D87400121CAA1200D0020ED822D282121C6F7402121CAA96
:201D4B00D2837F0212223CC283121CA80C121C74C282121C3D502020BC17201214D28212AB
:201D6B001C6F7402121CAA121C4AD28312223CC283121CA8C28222121CBD80BAD283121C19
:201D8B006FD2827404121CAA12307B121CA8C283C2820C121C74121C3D502020BC1520125D
:201DAB0012D283D282121C6F7404121CAA121C4A12307D121CA8C283C28222121CBD80BC91
:201DCB00C284D283121C6F121CA4C284123071121CA8121C74C2830C121C3D501A20BC116A
:201DEB0020120ED283121C6F121CA4121C4A123073121CA8C28322121CBD80C4C2BCD28368
:201E0B00D284121C6F121CA4123085121CA8C283C2840C121C74121C3D501B201210D283AF
:201E2B00D284121C6F121CA4121C4A123087121CA8C283C28422121CBD80C1C2BCD283D23D
:201E4B0084121C6F7408121CAA123085121CA8C283C2840C121C74121C3D501D201212D23E
:201E6B0083D284121C6F7408121CAA121C4A123087121CA8C283C28422121CBD80BDC2BC23
:201E8B00D284D2A4D2A0121C6FD280C2A4121CA4123071121CA8C2840C121C74121C3D509A
:201EAB001920120ED284121C6F121CA4121C4A123073121CA8C2A4C28422121CBD80BFC23C
:201ECB00BCD284D2A4121C6F121CA4123067121CA80C121C74C284C2A4121C3D501B20121F
:201EEB0010D284D2A4121C6F121CA4121C4A123069121CA8C284C2A422121CBD80C1C2BC1B
:201F0B00D284D2A4121C6F7410121CAA123067121CA80C121C74C284C2A4121C3D501D2020
:201F2B001212D284D2A4121C6F7410121CAA121C4A123069121CA8C284C2A422121CBD807B
:201F4B00BDC2BCD290C2A5C2B5D2B3D2A4D285D294BA0A0A301F05D291021F69D295121C9F
:201F6B006F1227C512283475F020121C9B7F0EDFFE123067201E0675F000121C9B0C121C6E
:201F8B0074BA0A187E00301F0B20911012176DDEF8021FA720950512176DDEF8C2B3C29428
:201FAB00121C3D502A201217D294D2B3121C6F75F020121C9B7F0EDFFE121C4A1230691273
:201FCB001CA81227C5122834C294C2B3C29522121CBD021F4C120F04121C6F75F020121CB5
:201FEB009B7F0EDFFE431F801228447F0412223C531F7F1228447F0EDFFE121CA87F0EDF63
:20200B00FE121C74120EF00C121C3D500A1227C5122834121CA822F52E85F02FC29412277A
:20202B00C5122834121CA8BC0303021CC880A6742375F01812206474201220647422122022
:20204B0064741875F004122064741B1220647419122064741A12206422122618E5F012269B
:20206B0039C2A4C284121C51D284D2A422C2BCD284D3920C122834D2A4D2A0D280BA191A29
:20208B007E10121C76122A7C121C60121C6F122A7C7F28DFFEC2A4C28422BA0F4F301F0DA2
:2020AB001228B3D2807401121CAA0220C5301D0A1228B3D2847410121CAA122A68121C607A
:2020CB00121C6F122A7C7F10DFFE121C74301D0AC2A4C3920C12283401E9C2A4C284121C42
:2020EB003D4003021CC37400121CAA22D280BA1111301F04D2842105D2A17411121CAA0237
:20210B002110121CA47E40121C76122A7C121C6F122A7CBA1134121CA4D284301F1CC2A44A
:20212B00C3920C1228347F08DFFE121C51F5F0D3920C122834D2A4E5F022C2A4C2847F087E
:20214B00DFFE121C51D284D2A4227F14DFFE7EC0121C76122A7C7F10DFFE121C74C2A4C2EA
:20216B00840C121C3D5010D284D2A4121CA87F08DFFEC2A4C28422121CBD0220781228A1C5
:20218B00122897121C747E00BA0B33D28100D28200C283121C608EF0121C76C28100D28119
:2021AB00121C74C28300C282121C51B5F051AEF00ED2821228523010DAD283020F22BA0C80
:2021CB0036D2A0D283C284121C608EF0121C76BA0C02D2A1D2A0C2A0D2A0121C74C283C2D7
:2021EB0084121C51B5F018AEF00ED2831228523010D5D284020F22BA0D0280C5020F2202A6
:20220B001CC37B0212007F04F527FE752600782B12007FF62526F52608DEF512007FB52636
:20222B00067455120092227401120092DBD6020033120012BF00FD22EEA2E09290A2E19256
:20224B0091A2E29292A2E392A5A2E492A4A2E59285A2E69284A2E792A322E5905407A2A58F
:20226B0092E3A2A492E4A28592E5A28492E6A2A392E722E519A2E092B2A2E19286A2E29291
:20228B0097A2E392DAA2E492B4A2E592D9A2E692D8A2E79280E51AA2E092A0A2E192A1A255
:2022AB00E292A2A2E39215BA0104A215928122EEA2E09292A2E19293A2E29294A2E392B574
:2022CB00A2E492B3A2E592A5A2E692A4A2E7928522A29292E0A29392E1A29492E2A2B59209
:2022EB00E3A2B392E4A2A592E5A2A492E6A28592E722E519A2E09291A2E19290A2E292B2D7
:20230B00A2E39286A2E49297A2E592DAA2E692B4A2E792D9E51AA2E09281A2E19282A2E202
:20232B0092A3A2E392A2A2E492D8A2E592A1A2E69215A2E79216BA1E17201F0AA215928099
:20234B00D392A002236CA21592A0D3928002236CBA0404A2169280BA020302236CA2159258
:20236B00A022A2E09291A2E19290A2E292B2A2E39286A2E49297A2E592DAA2E692B4A2E7E8
:20238B0092D922A2E09281A2E19282A2E292A3A2E392A2A2E492D8A2E592A1A2E69280D3F0
:2023AB0092A022EEA2E09294A2E19295A2E29296A2E392B6A2E492B7A2E592B5A2E692B39B
:2023CB00A2E792A522A29492E0A29592E1A29692E2A2B692E3A2B792E4A2B592E5A2B392C1
:2023EB00E6A2A592E722F590EEA2E692B3A2E792B5543FF5A022E590FEE5A0A2B392E6A249
:20240B00B592E7CE22E519A2E09293A2E19292A2E29291A2E39290A2E492B2A2E59286A2EE
:20242B00E69297A2E792DAE51AA2E092A2A2E19283A2E29285A2E392A3A2E492B4A2E59206
:20244B0082A2E69281A2E792D9BA1129301F1AD284E51BA2E092D8A2E192A1A2E2920FA244
:20246B00E3920D1228340224F3D392A1E51BA2E092D80224F3E51BA2E092D8A2E192A1A2F9
:20248B00E29215A2E39216BA240BA2E6920EA2E7920B0224B0BA250280F0BA0F20301E05E1
:2024AB00D2800224F3301D0ED284A215920FA216920D12283422A21592800224F3BA100703
:2024CB00A21592800224F3BA1907A21592800224F3BA0704A2169280BA05030224F3BA0926
:2024EB00030224F3A21592A022C2B2D2B3F590EEA2E692B6A2E792B7543FF5A02274FFF5EA
:20250B0090C2B2C2B3E590FEE5A0A2B692E6A2B792E7CE22D2B2E519F59012176DD28512A7
:20252B00176DC285E51AF59012176DD28612176DC286BA2624E51BA2E092D8A2E192D9A2F5
:20254B00E292DAA2E39282A2E49283A2E5928174FFF590C2B212176D22E51BA2E092D8A2A2
:20256B00E192D9A2E292DAA2E39281A2E49283A2E5928074FFF590C2B212176D22E51975B1
:20258B002100A2E092D8A2E192D9A2E292B4A2E392DAA2E4920CA2E5920DA2E692B2A2E7DB
:2025AB00920F122834D2B6C2B6E51A752100A2E092D8A2E192D9A2E292B4A2E392DAA2E451
:2025CB00920CA2E5920DA2E692B2A2E7920F122834E51BA2E09215A2E192167400A21592B7
:2025EB000BBA140BA216920E8521F012283422D380F4E51BA2E09215A2E192167400A215A8
:20260B0092E3BA1405A21692E622D380FAA2E09293A2E19292A2E29291A2E39290A2E49214
:20262B00B2A2E59286A2E69297A2E792DA22A2E092A2A2E19283A2E29285A2E392A3A2E44D
:20264B0092B4A2E59282A2E69281A2E792D97400A2E092D8A2E192A1A2E39216BA0F0830BB
:20266B001E05D280022676A216928022EEA2E092A0A2E192A1A2E29281A2E39282A2E492B0
:20268B00A2A2E59283A2E692A3A2E7928422E5A05403A28192E2A28292E3A2A292E4A28388
:2026AB0092E5A2A392E6A28492E722E519A2E09280A2E192D8A2E292D9A2E392B4A2E492C9
:2026CB00DAA2E59297A2E69286A2E792B2BA3B0302276FBA380302279FBA2C0E752100E53C
:2026EB0024A2E0920BE51A0226FAE51A752108A2E0920CA2E1920DA2E2920EA2E3920FA2A0
:20270B00E492B6A2E592B7BA120302271BBA200DA2E692B5A2E792B34408022769BA360D40
:20272B00A2E69295A2E792964408022769A2E6921630BA06A2169291E15DA2169295F5F053
:20274B00E51B5480B48009E5F0A2E79296022769E5F04408301E07446054F802276B54F8FF
:20276B0012283422301F0675210002277B752108E51AA2E0920CA2E1920DA2E2920EA2E3A7
:20278B00920FA2E492B6A2E592B7A2E692B5A2E792B380CAE51AA2E0920CA2E1920DA2E243
:2027AB00920EA2E3920FA2E492B6A2E592B780AEA2E69295A2E7929680A4E51A752108A2B9
:2027CB00E0920CA2E1920DA2E2920EA2E3920F221227C5122834221227C55321F71228347D
:2027EB0022E51B752110A2E2920FA2E3920D221227EC5321EF122834221227EC43211012D8
:20280B00283422121C74749BF51F122846121CA8740012283675808075900075A0C075B0BC
:20282B000375D808C2BAD29922E5214401122AAEC2A6D2A7C287D28722E51F122AAED2A6EC
:20284B00D2A7C287D28722E51CB5190DE51DB51A08E51EB51B03D21022C3E5192401F519AD
:20286B00E51A3400F51AE51B3400F51BBA1B067406123BC02222E5255480700AE51F440180
:20288B00F51F12284622E51F54FC80F4431F04122844121C8522ED902AEB93F51F1228463D
:2028AB0022E5255430B40009E51F54E544080228CFB42007E51F54E50228CFB4100CE51F39
:2028CB0054E54410F51F12284622E51F54E54402F51F12284622BA2406201C38022909BA2B
:2028EB002503022909BA0F2C301C1374AA12261874021226397E55121C76122A7C22301D2A
:20290B0013745512261874051226397E55121C76122A7C2274AA122618742A1226397E55F5
:20292B00121C76122A7C227E000229967E200229967E900229967E400229967E6002299683
:20294B007EAA0229967EA00229967E800229967E100229967EA0121C76122A7C227EAA02D0
:20296B0029857EA002298574AA12236D742A12238E7E551222BA122A8522745512236D742C
:20298B005512238E1222BA122A8522BA2406201C340229BCBA25030229BCBA0F28301C11F1
:2029AB0074551226187405122639121C76122A7C22301D1174AA122618740A122639121CA2
:2029CB0076122A7C2274551226187455122639121C76122A7C2212294B1228E11229551288
:2029EB00294B1228E122122A01122A13122A25122A01122A1322751955751A551222FD7E0A
:202A0B00AA1222BA122A85227519AA751A231222FD7E551222BA122A8522751955751A55AA
:202A2B001222FD7E801222BA122A8522751955751A551222FD7E101222BA122A8522301DE7
:202A4B00012212296812297212296D2212293C1229322212294B1228E112293722BA250311
:202A6B0002295F12294B1228E112295022301DF322C2A4C2A0D2A0D2A422C284301F07C2E1
:202A8B0080D280022A95C2A0D2A0D28422C283C281D281D28322EA23F993C9A3938983F561
:202AAB0082E473C2A6C2A73392DBC287D2873392DBC287D2873392DBC287D2873392DBC239
:202ACB0087D2873392DBC287D2873392DBC287D2873392DBC287D2873392DBC287D28722E1
:202AEB003B5B9B1B0E410EA50E460E580EA50E460E580EA50E660E460E660E410E460E4670
:202B0B000E660E460E460E460E5D0E460E4615A645503EA10E460E4639B73DFF39B70E41E5
:202B2B000E460E464A0F4D6D4EC80E460E460E4607573B5E396B3B5E31FE55BB4AF236FFD9
:202B4B0008A30757425842584258425831FE4EC847BF32D046F1417907DA48F20A3E0B4FFE
:202B6B000CCC0FF90FF90FF91005101510371061107310A410A410A410A410A410A410A4F9
:202B8B0010A410A410A410A410A410A410A410A410A410A410A436A13E3036A110A410A4EA
:202BAB0010A44A764E114F5110A410A410A414F73B20398A3B2031CF52FC4C5C38920961CD
:202BCB00144544BE44BE450644BE31CF4F87486733C7486744BE1445495B0B1D0C8E0DCA7A
:202BEB00199419D1199919A619D1199919A619D119B3199919B319941999199919B31999A4
:202C0B002E43199919AB17981798162445C13F47177C1999365A3DA436272DA42E031999D7
:202C2B004A884DA24ED91CDB1CDB1CDB1B8B3A9F39B63AD2314E53984BF83769091419F5CA
:202C4B00431F43D0443042DF31884ED9489734A6489741F01B0A49860AD00C410D880FF502
:202C6B000FF50F380F380F380F420F420F420F850F420F850FF50FF50FF50F850F420F42C2
:202C8B000F420FF50FF50FF50FF50FF50FF503520F420FF50FF50FF50FF50FF50FF50F856E
:202CAB000F420F420F420F420F4209940FF50FF50FF50FF50FF54B450FF509940994099458
:202CCB000994099409940FF50F42480F0FF5480F099409940F850994099409941D411D8764
:202CEB001DCB1E071E461E891ECA1F091F4C20781F4C1D401D401D401F4C207820782078E9
:202D0B001FE0207820781D401D401D401D4020781D401D401D401D401D401D401D4020784A
:202D2B00207820782078207820781D401D401D401D401D401D401D401D40207820782078E0
:202D4B00207820781D40207820781D402078207820781D401D401D401D400000010101020D
:202D6B00020203020300010103020202030202020202020203030300010203020202020207
:202D8B00020303030303030302020202020203020303030203030202021200D012220DD2F4
:202DAB0081D282D283782B121C60121C6F122A987B02121C9212285208D527EB1200D03072
:202DCB0010DA020ED81200D012220DD283D284D2A0D2A1782BE6FE081222FD122A851222AE
:202DEB00BA122A857F0612223C122852D527E61200D03010D3020ED8301C0280C8D283D250
:202E0B0084301F04D280C115D2A01200D012220D122A49782BE6FE081222FD122A851222D9
:202E2B00BA122A85122852D527EB7F3C12223C3010CB1200D0020ED8D2A4D2A0D284120049
:202E4B00D0301E2B12220D122A78782BE6FE08122410122A7C1223AE122A7C122852D52779
:202E6B00EB7F1412223C3010CF1200D0020ED8752600122EBE50FB0E8E27122A78122EBE27
:202E8B004005122A7C80F62526F526122410122A7C1223AE122A7C122852D527E012007FBC
:202EAB007F1412223C745512009230108B1200D0020ED8C3309806D3E599FEC2982212286C
:202ECB00A1122897C2BCD284D2A4D2A01229E1122941122410AE1C1223AE122A7C7F1412D1
:202EEB00223C020ED87B28121C92743112009222121C74BA2103024DDABA2203024FC0BA60
:202F0B003503024FC0BA2603022F49BA2F03022FA0BA3A03022FA01228A1122897D284D2A7
:202F2B00A4D2A012294B1228E112293C7B28121C92121C74121C60C2A4C284020FE11228ED
:202F4B00A1122897D280D2B4D2B2D2B3D2840000C2840000D28412176D12176D12176D124D
:202F6B00176D12176D12176D74907E001224F4C2B2C2B400D2B4D2B212251F12250812004F
:202F8B0092F526EE1200922526F52612009212007F12280E221228A1122897D2B4D2B2D25A
:202FAB00B3D2840000C2840000D28412176D12176D12176D12176D12176D12176DC019C044
:202FCB001AC01B7400F51B74057E557FAA12158F74027EAA7F5512158F74057E557F9012AD
:202FEB00158FD01BD01AD01912251FC2B4C2B200D2B4D2B212176D122508120092F526EE98
:20300B001200922526F52612009212007F12280E22BA0F02800302304B1228A11228971273
:20302B001C601228B3D283D2847418121CAAD2A4D2A0C2A4C2A07F1412223CD2A0020ED800
:20304B001228A1122897C2BCD284D2A4D2A01229E11229377F1412223C020ED87F01C2A49E
:20306B0012223CD2A4227F01C2A012223CD2A0227F01C28312223CD283227F01C2841222B1
:20308B003CD28422E52612009212007F221200922526F526122852221200922526F526222B
:2030AB007A083392810012176D12176DA2A1D2A012176D12176D00C2A0DAE733D281221253
:2030CB00280E121C90121C901228A1C2A0C280122897D28012176D12176DC280D2A1752615
:2030EB0000C217C2127B50121C9274AC1230AB74531230AB74001230ABF5F01230ABE5F0C4
:20310B0022E51B201C07C3301201D392E31230ABE51A1230ABE5191230AB22E608F525857E
:20312B001B18531BBF431B2012310C1230AB85181BB525012212310CE5251230AB7B1412CE
:20314B001C92221230CA1200D012220D201F03121774782BC212123126201F05D21212313B
:20316B0026122852D527ED1200D03010DC020ED8E608F52512310CE5251230AB22201FC351
:20318B001230CA1200D012220D851A28851929121774782BC21212317BD21212317B1228B9
:2031AB0052D527F0744C1230ABE5281230ABE5291230AB1230AB7B14121C921200D03010C6
:2031CB00C5020ED8C2131230CAE51B1230ABE51E1230AB74001230ABE51A1230AB7B50124F
:2031EB001C921200D012280E2212310C1230AB1230A3221230CA2013CBC2121231F4201C36
:20320B0008201F05D2121231F41228523010EA12308F12280E221228A17440121CAAC280A2
:20322B00431F041228447F28DFFEC2D87A0300D2D800C2D800DAF7C281C2A1C2A01228B3FA
:20324B00121CA47F14DFFED2A07FC8DFFE7FC8DFFE7FC8DFFEC2D8752600C21222C3928142
:20326B0092A1D2D800C2D87A08C0E0E5F03392A1F5F0D0E033928100A2A0D2D800C2D8000E
:20328B00DAE7E5F033C3928192A1D2D800C2D800C3928192A1D2D800C2D822E51B201C075B
:2032AB00C3301201D392E375F04C123268E51A75F04C123268E519123268221232A6123202
:2032CB00681230A3221232213013030233C730170302333275F04C7402301F02240112323B
:2032EB006875F00CE51912326875F01CE51A12326875F068740012326875F06C740012329E
:20330B00681230A3201F1375F078740012326875F07C74001232681230A31228523010C193
:20332B0012308F12280E22C217201D5375F04C7404123268E51A20E323301B1075F0787438
:20334B000012326875F07C74000233BA75F068740012326875F06C74000233BA301B107581
:20336B00F07A740012326875F07C74000233BA75F06A740012326875F06E74000233BA75DA
:20338B00F04C740812326875F00CE519123268301B1075F078740012326875F07C740002F4
:2033AB0033BA75F068740012326875F06C74001232681230A312308F12280E2220132D12A5
:2033CB0028A112289712322175F04C748012326875F064740012326875F06C7400123268B8
:2033EB007B64121C921200D012280E22C213E51E20E66F20E34920E22375F04C7440123270
:20340B006875F02CE51A12326875F064740012326875F06C740012326802348D75F04C743B
:20342B004012326875F02CE51A12326875F066740012326875F06E740012326802348D7543
:20344B00F04C744012326875F02CE51A12326875F074740012326875F07C7400123268028D
:20346B00348D75F04C742012326875F02CE51A12326875F064740012326875F06C74001213
:20348B0032687B14121C9275F04C74001232687B14121C921200D012280E22123221120055
:2034AB00D012220D851A28201F03121774782B75F04C7410301F02240112326875F00CE5FA
:2034CB001912326875F02CE612326808301F1375F06D740012326875F06C740012326802AA
:2034EB00350575F03CE60812326875F07D740012326875F07C7400123268122852D527BC05
:20350B00201F0875F01CE52812326875F064740012326875F06C74001232687B14121C92F6
:20352B001200D02010030234AC020ED8222020207A0833928312176D12176D0000A2A3D212
:20354B008412176D12176D00C284DAE633D283227A0833928312176D12176D0000D28412A2
:20356B00176DA2A312176D00C284DAE633D2832212280EC220E51854C0B48007D220D211E6
:20358B00121CAA121C90121C901228A1C284C2851228977B50121C9212176D12176DD28585
:2035AB007B50121C92202002C285D2A3752600C217C21274AC1235387453123538740012C4
:2035CB003538F5F0123538E5F022E51B20200A201C07C3301201D392E3123538E51A123578
:2035EB0038E51912353822E608F525851B18531BBF431B201235D512353885181BB5250150
:20360B00221235D5E5251235387B14121C9222E608F5251235D5E5251235382212357B12C4
:20362B0000D012220D201F06202003121774782BC2121235F2201F08202005D2121235F2F0
:20364B00122852D527EA1200D03010D6020ED8201FCA12357B1200D012220D851A288519BA
:20366B0029121774782BC21212361AD21212361A122852D527F0744C123538E52812353817
:20368B00E5291235381235387B14121C921200D03010C5020ED8C213C21712357BE51B1273
:2036AB003538E51E1235387400123538E51A1235387B50121C921200D012280E221235D5AC
:2036CB001235381230A322C291C280C286C2B2C290C2851228B3121CA47F14DFFE7FC8DF1A
:2036EB00FE7FC8DFFE7FC8DFFEC2DAD286D2D9C2D8D297221236D23013030238B2C290D245
:20370B0085C2B2301702C217E51B546F123888C29000C285D2B2E51A123888C2B2E519127C
:20372B00388874FF12071DC2B2C297301C04D2D8D2851238671200922526F526C297D2B25F
:20374B00123867D297201F071200922526F5261228523010BAE52612009212007F221236C4
:20376B00D2201B69C290D285C2B2E51B547F1238881200D012220D201F03121774782B124F
:20378B00379C122852D527F71200D03010E6020ED8C290C285D2B2E51A123888C2B2E5197C
:2037AB00123888D290E608123888C290C286D28612385C201F16E608D290123888C290D2D7
:2037CB00B2C286D28612385CC290C2B222E51B54F7F51BC290D285C2B2C2B4E51B547F122B
:2037EB0038881200D012220D201F03121774782B851A2A123836122852D527F7C290C285F8
:20380B00D2B2E52A123888C290C2B2C286D28612385CC290C2B21200D03010C9C290D285D2
:20382B007400123888121C90020ED8C290C285C2B2E519123888D290E608123888201F0B48
:20384B00D2B2E608D290123888D2B2D2B400C2B422D2D974FF12071D30D9F622A28492E008
:20386B00A2A392E1A28392E2A2A292E3A28292E4A28192E5A2A192E6A2A092E72212071D31
:20388B00D2DA0000C2DA221228A11228971236D2C290D285C2B27480123888C286D2867BEF
:2038AB0028121C92021441C213C290D285C2B2E51B54FC123888D290C285E51E12388830FC
:2038CB001909C2B2D2D8D2850238E8301809D2B2C2D8C2850238E8C2B2C2D8C285C286D2DD
:2038EB00867B14121C9202144112280EC220D211121CAA121C90121C901228A1122897C2C2
:20390B0084C282C28512176D12176DD282D2857B14121C92D2A3C282752600C217C21274F2
:20392B00AA12353874AC12353874531235387400123538F5F0123538E5F0D2822274AA129C
:20394B0035387438123538E51A123538E51912353822C282123948123538D2821230A322F6
:20396B001238F430130302398A30170302398A12395D1228523010F712308F12280E22C27C
:20398B0013C2171238F474AA123538E51B123538E51E1235387400123538E51A1235387B68
:2039AB0050121C921200D012280E222212357B3013030236A13017030236A1C2121236C896
:2039CB00201C0B201F08202005D2121236C81228523010E712308F12280E227A0833929749
:2039EB000000A286D2B200000000C2B2DAEF33D29722C220E51854C0B48002D22012280EB2
:203A0B00121C90121C901228A1C2B2C2901228977B28121C92D29012176D12176D2020027A
:203A2B00C290D286752600C217C21274AC1239E674531239E674001239E6F5F01239E6E5A0
:203A4B00F022E51B20200A201C07C3301201D392E31239E6E51A1239E6E5191239E622E6D6
:203A6B0008F525851B18531BBF431B20123A4D1239E685181BB5250122123A4DE525123949
:203A8B00E67B14121C9222E608F525123A4DE5251239E6221239FD1200D012220D201F0616
:203AAB00202003121774782BC212123A6A201F08202005D212123A6A122852D527EA120044
:203ACB00D03010D6020ED8E51854C0B4C0C6201FC31239FD1200D012220D851A28851929C7
:203AEB00121774782BC212123A92D212123A92122852D527F0744C1239E6E5281239E6E57B
:203B0B00291239E61239E67B14121C921200D03010C5020ED8C2131239FDE51B1239E6E5BE
:203B2B001E1239E674001239E6E51A1239E67B78121C927B78121C927B78121C927B781238
:203B4B001C921200D012280E22123A4D1239E61230A3221239FD2013BCC212123B54201CA7
:203B6B000B201F08202005D212123B541228523010E712308F12280E22E5197005E51A704E
:203B8B000122851A1D85191C751A00751900122852201009D2DA0000C2DA3010F1C21085CF
:203BAB002D1B852D23852E1A852F1985301E85311D85321C22201E0E7906543F139290D243
:203BCB0091C291D9F7227906543F1392A0D2A1C2A1D9F722201E2E7908D290D2910000C271
:203BEB009100D2910000C291A29013D9F5F5F07906D2910000C291A29013D9F5D2910000D0
:203C0B00C2910000227908D2A0D2A10000C2A100D2A10000C2A1A2A013D9F5F5F07906D22C
:203C2B00A10000C2A1A2A013D9F5D2A10000C2A1000022201E2F7908C290D2910000C29164
:203C4B00139290D2910000C291D9F57906E5F0139290D2910000C291D9F5C290D2910000DE
:203C6B00C291D290227908C2A0D2A10000C2A11392A0D2A10000C2A1D9F57906E5F01392C7
:203C8B00A0D2A10000C2A1D9F5C2A0D2A10000C2A1D2A02275F004E523540125F0123BC021
:203CAB00123BDF0303201B03543F22540F22122897201E07C291C290023CCAC2A1C2A012B5
:203CCB0028B3121CA4301914201B197400123BC0743FF5F074FF123C3E023CEF301B057472
:203CEB0006123BC022C212123C9F201803B51808E5F0B52503023D05D21222123C9FF52EA7
:203D0B0085F02F752705752B00851A2C85192D12009A020033201B0775F019E5F0A12F7562
:203D2B00F00B74089BA4FB227402123BC0E5258518F0123C3E7408123BC07F64DFFE740E34
:203D4B00123BC022201B057B19023D597B08123D33123CF0301204DBF580A0123D20DBC832
:203D6B002275F002E523540125F0123BC0E5258518F0123C3E301F0D20180A201907E51931
:203D8B005407B407137408123BC07B28121C92123CF0301203023D0622123CB9123B84122F
:203DAB0000D012220D201803121774782B30180574FF023DC2E608F518201B0553183FA125
:203DCB00CF53180FE6F52508301F08201805201902A1E7123CF030120B301A05123D6CA1FA
:203DEB00EF123D4F122852D527C31200D03010B2020ED822123CB9123B84752600123C9FA2
:203E0B002018071200922526F526E5F01200922526F5261228523010E4E5261200921200FE
:203E2B007F12280E22123CB9301C1B7409123BC07B28121C92740B123BC07B28121C921232
:203E4B0000D012280E22301F11741F123BC07B28121C921200D012280E227F077406123B21
:203E6B00C0DFF97402123BC0743FF5F074FF123C3E7401123BC07407123BC07408123BC0F2
:203E8B007B28121C927401123BC07407123BC01200D012280E227404122836201805C2A1D6
:203EAB00023EB3201944D2A1D2B4C280D280752600C217C21275F060123FEE7400123F36B3
:203ECB0030180A1200922526F526123F36C280120092D2802526F5261228523010D7E526A8
:203EEB0012009212007F12280E22D2A0D2B4C280D280752600C217C21275F060123FEE74CC
:203F0B0000123F361200922526F526123F36C280120092D2802526F5261228523010DAE555
:203F2B002612009212007F12280E2279083392D900D2D800C2D8A2B4D9F333227404122825
:203F4B00361228811228971200D012220D301803121774201805C2A1023F6B20193DD2A154
:203F6B00D2B4C280D280782B1240C275F050123FEEE608123F36301805E608123F36C2D99F
:203F8B0000C28000D2800030B4FDD2D9122852D527D61200D03010B2020ED8D2A1D2B4C221
:203FAB0080D280782B1240C2D2A0D2B4C280D2801240C2C280D28074507904123F38E62069
:203FCB001D057906023FD47908123F38C2D900C28000D2800030B4FDD2D91228521200D0ED
:203FEB00020ED8E51BC4540F903FF9022AA24003402340424060408DE5F07904123F38E5BC
:20400B00193333301207448054BF02401D30170244C07906123F3822E5F07904123F38E560
:20402B001933301207448054BF02403C30170244C07907123F3822E5F07904123F38E5193A
:20404B00301207448054BF02405A30170244C07908123F3822E5F0E51AA2E0E5F092E385FB
:20406B0019F0301208440853F07F024080301705440843F0807905123F38E5F07908123F19
:20408B003822E5F0E51AA2E19215A2E09216E5F0A21592E3A21692E28519F0301207440843
:2040AB0054FB0240B5301702440C7906123F38E5F07908123F382275F040C212D217123F5A
:2040CB00EEC280C217D28022D2A1D2B4C280D2801240C2D2A0D2B4C280D2801240C2747033
:2040EB007904123F3874FF201D0579060240FC7908123F38C2D9C280D28030B4FDD2D9C2B6
:20410B0012021441D2D87908C2A10000A2D83300D2A1D9F422C280740112465F7400124654
:20412B005F000000C2A100D2800022C280740512465F12410FD28020E0F122C280745012ED
:20414B00465F00C2A100D280C280740112465F740012465F000000C2A100D2800022C28048
:20416B00740512465F12410FD28020E0F12212423F752600AB1DAC1CEC60010BC212C28011
:20418B001241AA12410F1200922526F526DCF4DBF2D280E52612009212007F12280E22749E
:2041AB00E812465FE51B12465FE51A12465FE51912465FE51912465FE51912465FE51912B9
:2041CB00465FE51912465F22E51B12465FE51A12465FE51912465FC3E51A251EF51AE51B22
:2041EB003400F51B2212423F1200D0AD1EC280748212465F1241D312220D782BE6081246CF
:20420B005FD527F8E51C14700BD28012422F1200D0020ED8F51CDD07D28012422F80C912EC
:20422B0000D080D3C280745712465F12410FD28030E7F1227440D211121CAA122897C2B4F8
:20424B00C2BCD212D2D8D280D2A0D2D92212423F752600C212E51830E6121246D4C28074AD
:20426B00C512465F740112465FD28000C2801242B520141E12410F1200922526F5261228F6
:20428B00523010F0D280E52612009212007F12280E2212410FB4FF0C1228523010F41200A2
:2042AB00D0020ED61200DA020ED6301712C217E51920E10574900242CC740512465F22745B
:2042CB000312465FE51B12465FE51A12465FE51912465F2212423F1246D41241201200D0C1
:2042EB0012220D782B1246D47402C28012465F1242CFE60812465FD280C280740512465FA8
:20430B0012410FD280122852D527DA1200D03010CF020ED812423FE51820E74F30E6121283
:20432B0046D4C28074C512465F740112465FD280001200D012220D782B1246D47402C280FE
:20434B0012465F1242CFE60812465F122852D527F5D280C280740512465F12410FD28020BE
:20436B00E0F11200D03010CC020ED81246D4124120301F0A7B78121C927B78121C9212001B
:20438B00D012220D782B1246D47402C28012465F1242CFE60812465F122852D527F5D2802C
:2043AB00C280740512465F12410FD28020E0F1301F0A7B78121C927B78121C921200D0300A
:2043CB0010BF020ED812423F1246D41241201200D012220D121774782B1246D474ADC280F7
:2043EB0012465F1242CF61FA74ADC28012465FE60812465F122852E60812465F122852D22F
:20440B0080D527E47404C28012465FD280C280740512465F12410FD28020E0F11200D03045
:20442B0010AF020ED812423F1246D41241461200D012220D782B1246D474AFC28012465F64
:20444B001242CF815774AFC28012465FE60812465F122852D280D527EC121C907404C28057
:20446B0012465FD280C280740512465F12410FD28020E0F11200D03010B7020ED87405C215
:20448B008012465FD280227450C28012465F00C2A100D280227401C28012465F7400124698
:2044AB005F00C2A100D280221244885403B4030280F62212423F7F1412223C1246D4124120
:2044CB0020121C90121C90121C901246D4C28074C712465F0000C2A10000D280121C901292
:2044EB001C90121C90C280740512465F12410FD28020E0E80214411200DA2212423F7F14AE
:20450B0012223C1246D41244921244A01244B31246D4C280746012465F00C2A100D280124D
:20452B0044B31244921244A01244B31246D4C28074C712465F00C2A100D2801244B302145E
:20454B00411200DA22201A37D2D8D280D2A0D2D9C2B4752600C217C21275F003C2801246B7
:20456B006D12410FD2801200922526F5261228523010E6E52612009212007F12280E22D2D7
:20458B00D8D280D2A0D2D9C2B4752600C217C21275F003C28012466D12410FD28012009244
:2045AB002526F5261228523010EEE52612009212007F12280E22201A54122881122897D23A
:2045CB00D8D280D2A0D2D9C2B41246D41241201200D012220D782B1246D4C28075F00212C7
:2045EB00466DE60812465FC2A10000D2800000C280740512465F12410FD28020E0F1122852
:20460B0052D527D31200D03010C8020ED8122881122897D2D8D280D2A0D2D9C2B41246D455
:20462B001241201200D012220D782B1246D4C28075F00212466DE60812465F122852D5276F
:20464B00F5C2A1D2807B28121C92003010C51200D0020ED8790833C2A100928133D2A1D9CA
:20466B00F622E51BC4540F904678022AA24682468D469846A946C4E5F012465FE519124680
:20468B005F22E5F012465FE51912465F22E51AA2E0E5F092E312465FE51912465F22E51AD3
:2046AB00A2E0E5F092E3F5F0E51AA2E1E5F092E412465FE51912465F22E5F012465FE51A58
:2046CB0012465FE51912465F22C280740612465FC2A100D28022D290C2A5D2A4D285D291FE
:2046EB007FC812223C221246E1301703024743301303024824C2B5D2B330180EC294431F09
:20470B0080122844752100024720D294531F7F122844752108121C60C2B3121C51D2B31205
:20472B0000922526F5261228523010E9E52612009212007F12280E22C217D294C2B5D2B3DC
:20474B00431F80122844752100121C6000C2B300020FE1D290C2A5D2A4D285431F801228B1
:20476B0044751930121C601227E2121C517F0312223C124787852F19852E1A22D2A4D2B579
:20478B00C2B3431F80122844D294E51B5401B40106751AA50247A5751A55121C60121C768B
:2047AB00C2A47F06DFFE00D2A47E0020940512176DDEF82212475E30170302480F3013034B
:2047CB00024824C2B3C2B5531F7F122844121C90121C60121C5130140CB4FF030247F712E2
:2047EB0000DA020ED61200922526F5261228523010DE301403020F22E52612009212007F80
:20480B0012280E22C217C2B3C2B5431F80122844121C601227E2020FE1C213201B10D2B5BC
:20482B00D2B3431F801228441227E202484EC2B5C2B3431F80122844D294751A55121C60B1
:20484B00121C76D294C2A47F06DFFE00D2A47E0020940512223CDEF81200D02212109A12B6
:20486B001C9012475ED2A4D2B5C2B3431F801228441227E2D294C2A47F06DFFE00D2A47EBB
:20488B0000209405121C92DEF802144112475ED2A4C2B5D2B3531F7F1228441200D01222B9
:2048AB000D782BD294121C60121C6FC2A47F06DFFE00D2A47E0020940512176DDEF80812B1
:2048CB002852D527DE1200D03010D3020ED8C285C2A5C2A4D29043A0101228A11228977F08
:2048EB0004121C90DFFB221248D9752600121C74301F091227C55321F7122834531F7F431C
:20490B001F04122844301703024945D296D292D293C294C295D291121C60C291121C51D29E
:20492B00911200922526F5261228523010E7E52612009212007F12280E22C217D296D292CF
:20494B00C293C294C295D291121C60C291020FE11248D9431F80122844C296C295C293D2AB
:20496B0091D292D2947F0ADFFEC2927FC812223CC2947F78DFFED292021441C2101248D976
:20498B00301F091227C55321F7122834531F7F431F04122844C296D291C294D2921200D0B1
:2049AB0012220D782B121C60121C6FD2957F0ADFFEC2927F14DFFED2937F32DFFEC293C242
:2049CB00957F0ADFFED29212285208D527D71200D03010CC020ED8C285C2A5C2A4D2B3D2C5
:2049EB00B51227C5122834531F7F431F04122844D2907F04121C90DFFBC290121C90D285D2
:204A0B0043A030221249E2301703024A4F539000531F7F201F03431F80431F04122844D286
:204A2B0096121C60C296121C51D2961200922526F5261228523010E7E52612009212007F0B
:204A4B0012280E22C217539000E51920E009D291D292D294024A66D293D294431F04D296A6
:204A6B00122844121C60C296020FE11249E243906CC2957B3C121C92D2950214411249E290
:204A8B005390C0D296D291531F7F201F03431F80431F041228441200D012220D782B121CB0
:204AAB0060121C6FC2957F32DFFED29512285208D527EB1200D03010E0020ED8E51F448075
:204ACB00F51F122846D2A5D2B3D2947FFADFFE1228B375F020121C9BD290D2857FFADFFE35
:204AEB00C2A57F32DFFE22124AC7301703024B45301303024B63C291C292C220C2B5D2A429
:204B0B00C294121C60C2B3121C51D2B330140CB4FF03024B2D1200DA020ED61200922526EC
:204B2B00F5261228523010DA301403020F22E52612009212007F12280E22C217124AC7D2B7
:204B4B0091D292D220D2B5D2A4C294121C60C2B3121C51D2B3020FE4C213E51B5480B48037
:204B6B000BC291D292C220C2B5024BC3C291D292201B07D220C2B5024B89C220D2B57C00E2
:204B8B00121C60AE1BEE540FFE121C76C294C2A47F06DFFE00D2A40C121C74C2B3121C518A
:204BAB008EF0540FB5F00AD2B3D2941200D0020ED8D2B3121CBD80CB7C00121C60AE2B12F5
:204BCB001C76C294C2A47F06DFFE00D2A40C121C74C2B3121C51852BF0B5F00AD2B3D294C8
:204BEB001200D0020ED8D2B3121CBD80D0124AC7E51B5480B4800BD291C292C220C2B502D8
:204C0B004C15D291D292C220C2B57521001228341200D012220D782B7C00121C60121C6F97
:204C2B00C294C2A47F06DFFE00D2A40C121C74C2B3121C3D5014D2B3D29408122852D52768
:204C4B00D71200D03010CC020ED8D2B3121CBD80CC122897751B00751A00751900751E00CF
:204C6B00751D80751C00124AC7E51B5480B4800BD291C292C220C2B5024C8ED291D292C2DB
:204C8B0020C2B5752100122834124D25751B00751A00751900751E00751D08751C00E51B7F
:204CAB005480B4800BD291C292C220C2B5024CC3D291D292C220D2B5752100122834124D22
:204CCB0025E51B5480B4800BD291D292D220C2B5024CE6D291C292C220C2B575210012284D
:204CEB0034751B00751A00751900C294C2A4121C90121C90D2A4D294D291D292D220C2B584
:204D0B00752108122834C294C2A4121C90121C90121C90D2A4D2940214417C00121C607ECB
:204D2B0000121C76C294C2A47F06DFFE00D2A40C121C74C2B3D2B3D294081228523010DA74
:204D4B0022D2B3121CBD80D7D2A4D285D2A0D284D2D8D280D281C2D87F1EDFFED2D830A4E9
:204D6B00FD22124D537EFF1223AE124E47C2841223D0D2841200922526F5261228523010D9
:204D8B00E9E52612009212007F020ED81200D012220D782B024DAA124D531228B3782B12E4
:204DAB004E477E401223AEC285D285121CA4121C6FC285D2857F04DFFE30A4FD121CA808F8
:204DCB00122852D527D93010C31200D0020ED81228A1122897121C74124D53124E477E90E5
:204DEB001223AE000000C285000000D285000000C2840000001223D0D2841200921200923E
:204E0B0012007F020ED81228A1122897124D531228B3124E477E201223AEC28500D28512EB
:204E2B004E47121CA47ED01223AEC28500D2857F08DFFE30A4FD121CA8021441E519A2E04F
:204E4B009293A2E19292A2E29291A2E39290A2E492B2A2E59286A2E69297A2E792DAE51A1F
:204E6B00A2E092B4A2E192D9A2E292A1C2A0E51AA2E39293A2E49292A2E59291A2E69290B1
:204E8B00A2E792B2E51BA2E09286A2E19297A2E292DAA2E392B4C392D992A1D2A022D2A4CE
:204EAB00D285D2A0D284D281C2D8D2D87FFFDFFE7FFFDFFEC2D87F0ADFFED2D822124EA9A6
:204ECB00024D701200D012220D782B024EE71228A1122897124EA91228B3782B124F35121E
:204EEB004E47121C6FC28500D2857F03C284000000001223D0D2845480F5F0E65480B5F09C
:204F0B001008122852D527D43010B81200D0020ED8DFD9F52E85F02F752705851B2B851AC6
:204F2B002C85192D12009A020ED8C019C01AC01B7EAA124FFF7E5512500C7EA0124FFFD036
:204F4B001BD01AD019221228A1122897124EA9C019C01AC01B7EAA124FFF7E5512500C7EAC
:204F6B0080124FFF7EAA124FFF7E5512500C7E10124FFFD01BD01AD0190214411228A1128D
:204F8B002897124EA9C019C01AC01B7EAA124FFF7E5512500C7E80124FFF7EAA124FFF7E83
:204FAB005512500C7E30D01BD01AD01912501830A4FD0214411228A1122897121C74124E67
:204FCB00A9C019C01AC01B7EAA124FFF7E5512500C7E90124FFFD01BD01AD019124E47C231
:204FEB00841223D0D28412009212009212007FC211020ED8751955751A55751B0012501862
:20500B00227519AA751A2A751B00111822124E471223AEC285000000D2852212507A7400FD
:20502B007EAA1223F1C286C3920E122834D3920E122834D286227519AA751A2A751B001210
:20504B00258874007E551223F180DA12507A74007E801223F180CE12507A74007E101223FC
:20506B00F180C212507A74007EA01223F180B6751955751A55751B001225882212289720FF
:20508B001E07C291C290025098C2A1C2A01228B3121CA422201E0E7904540F139290D291E7
:2050AB00C291D9F7227904540F1392A0D2A1C2A1D9F722201E137903540F139290D291C229
:2050CB0091D9F7139290D291227903540F1392A0D2A1C2A1D9F71392A0D2A122201E0D7942
:2050EB0008D2910000C291A29013D9F57908D2A10000C2A1A2A013D9F5201E1D7908D2911B
:20510B000000C291A29013D9F5F5F07908D2910000C291A29013D9F5227908D2A10000C217
:20512B00A1A2A013D9F5F5F07908D2A10000C2A1A2A013D9F522201E1D7908139290D291AB
:20514B000000C291D9F57908E5F0139290D2910000C291D9F52279081392A0D2A10000C2F7
:20516B00A1D9F57908E5F01392A0D2A10000C2A1D9F522740012509F75F00EE51B543F12C7
:20518B005141740012509F75F06E74F8125141740012509F75F00EE51A12514174001250B9
:2051AB009F75F06E74F7125141740012509F75F00EE519125141740012509F75F06E74F627
:2051CB0012514122740012509F75F00EE51A125141740012509F75F06E74F71251417400A8
:2051EB0012509F75F00EE519125141740012509F75F06E74F612514122740012509F75F03C
:20520B000E743C125141740012509F75F06E74F8125141740012509F75F00E7400125141C9
:20522B00740012509F75F06E74F7125141740012509F75F00E7406125141740012509F751C
:20524B00F06E74F6125141740C12509F75F0007400125141740012509F75F08E74A61251F4
:20526B0041740012509FE51B543FB4302375F08C74A6125141740012509F75F0EF740012D5
:20528B005141740012509F75F0F874001251412275F09C74A612514122740012509F75F0AA
:2052AB008474A6125141740012509F75F08874A6125141740012509F75F00E74551251412C
:2052CB00740012509F75F06E74A7125141740012509F75F00E74AA125141740012509F7528
:2052EB00F06E74A712514122740912509F12510422125087740012509F75F08E74A612518F
:20530B0041740012509F75F08C74A6125141740012509F75F00E743C125141740012509F6C
:20532B0075F06E74F8125141740012509F75F00E7400125141740012509F75F06E74F712BA
:20534B005141740012509F75F00E7404125141740012509F75F06E74F6125141740C125074
:20536B009F75F0007480125141740012509F7400F5F0125141740012509F7B28121C9274C8
:20538B0000F5F01251411200D012280E221250873018030254AA12520412517E1200D012BC
:2053AB00220D782BE51B543FB430030254281251CF740D12509FE608F5F0E608C5F012518B
:2053CB0041740D12509FE608F5F0E608C5F0125141740D12509FE608F5F0E608C5F012518A
:2053EB0041740F12509FE608F5F0E608C5F012514174001250BE7B0A121C92201E05C29154
:20540B00025410C2A17400F5F01251417B08122852DBFB1200D0301086020ED822740F128F
:20542B00509FE608F5F0E608C5F012514174001250BE7B0A121C92201E05C29102544CC285
:20544B00A17400F5F0125141740012509F75F02A74F61251411818740F12509FE608F5F00A
:20546B00E608C5F012514174001250BE7B0A121C92201E05C291025486C2A17400F5F012C1
:20548B005141740012509F75F02A74F61251417B02122852DBFB3010841200D0020ED812DE
:2054AB0000D012220D782B1255A012556E740012509F75F00EE608125141740012509F75ED
:2054CB00F06E74A8125141740012509F75F08474A6125141125539740012509F75F0827417
:2054EB00A612514112551E740212509F1251045402B400F012176D740012509F75F0947482
:20550B00A6125141122852D527A01200D0301092020ED8740012509F75F05074A61251418A
:20552B00740012509F75F06E74F512514122740012509F75F00E7455125141740012509F1F
:20554B0075F06E74A7125141740012509F75F00E74AA125141740012509F75F06E74A7128F
:20556B00514122740012509F75F00EE519125141740012509F75F06E74A912514174001253
:20558B00509F75F00EE51A125141740012509F75F06E74AA22740012509F75F09E74A612CF
:2055AB005141740012509F75F09C74A61251412212508775260020181F12517E1252F312D3
:2055CB0000922526F5261228523010F0E52612009212007F12280E221255A012556E740012
:2055EB0012509F75F08074A6125141740012509F75F05074A8125141740012509F75F06ECA
:20560B0074F5125141740212509F74FF1251041200922526F5261228523010BFE52612006F
:08562B009212007F12280E22EA
:00000001FF
